:1000000000308A00122900000A108A100A118207A3
:1000100029340034303400343C30840000080319A3
:1000200023280230F800BF30F7006400F70B1528D2
:10003000F80B13289630F700F70B1C28000000007F
:100040006400800B112800340830BE02031C3328E2
:100050003E3084000310800C000803193328312837
:100060006400800B302800348316051183120515B7
:1000700064000130BC000C206330BE002420240842
:10008000BB00BB0803194628BB0341288316051192
:10009000831205113430AE000030AF008A11BF2941
:1000A00000340108801F5728A61F5F285928A61B67
:1000B0006828A608031D5F282502031C68288316EC
:1000C000851083128510831605108312051470287D
:1000D0008316051083120510831685108312851070
:1000E0000108801F7628A81F7E287828A81B87284B
:1000F000A808031D7E282702031C87288316851362
:100100008312851383160513831205178F28831610
:100110000513831205138316851383128513640058
:100120000230BD00F730BE002420BD0B922883169C
:100130000610831206101308930183161418A228C0
:1001400083129D2883121308A100831606108312C0
:100150000614211CB328BC30A400A601A501A801E7
:10016000BE30A700F328211FBD28A801A701A601C2
:10017000BE30A5004430A400F328A11CC828A83034
:10018000A400A6019630A500A801BE30A700F32860
:10019000A11ED3285830A400A8019630A700A601BC
:1001A000BE30A500F328211DDE289430A400A6014E
:1001B0009630A500A801BE30A700F328211EE9282B
:1001C0006C30A400A8019630A700A601BE30A5009F
:1001D000F328A11DF3288030A400A601BE30A5009D
:1001E000A801A700F3285130B5000030B6008A11ED
:1001F000BF290034831605118312051564000130F0
:10020000BC000C206330BE0024202408B900B908CB
:1002100003190C29B9030729831605118312051147
:100220008A115B2984011F308305703083168F008B
:100230001F129F121B0880399B0007309C001F1261
:100240009F121B0880399B001F1383121F179F17D3
:1002500083169F1383121F1494128316061186149B
:100260000612303083129400003083169400010887
:10027000C7390838810083129001723083168F00CD
:1002800005138312051383168513831285138316B2
:100290000510831205108316851083128510803097
:1002A000A400B801B701B808031D62293708633CF0
:1002B000031C6229FA281030BC000C20B70A03196D
:1002C000B80A5329A601A501A801A701A901AB01FC
:1002D0000830AA00AD01AC013430AE000030AF00F0
:1002E000B001B2010130B100B401B3015130B50029
:1002F0000030B600A0010030F80006389200FA3055
:100300008316920083128C100030F8000638920099
:10031000FA308316920083128C100310200DF70020
:100320000420F900013077070420FA0079088400DE
:100330000008F900840A0008F700840A0008F800A1
:10034000840A800A0008FA00031DA929840A800A89
:100350008403840A00087802031DC12977087A0201
:10036000031DC12984038001840A8001840AF91BCA
:10037000C129840A00088A008403000882008312CD
:100380000313A00A02302002031D8D29A0018C1C3A
:0E039000CB2983168B29C729FF30A0006300FC
:04400E00383FFC3FFC
:00000001FF
